:021B3200EFF8CA
:061B1400000000D8FB22D6
:061B1A00F07814021B1418
:10191900908000E521D2E0121B1A6403121B1A649D
:0B19290003121B1ADFEFC2E0021B1AC2
:10119400C243EE2F604A0ED3121969303A00908090
:1011A40000E521203A05D2E0121B1A6403121B1A2F
:1011B4006403121B1A203A05C2E0121B1AEFBE0187
:1011C40005C3940440045CB40112C3121969A93123
:1011D4007840121B14D9F9DFBEDEBC22DFC3DEC1A6
:0711E400908002E524F022D7
:10186F00EE2F601E0E908000E521D2E0121B1A644D
:10187F0003121B1A6403121B1AC2E0121B1ADFEAAF
:03188F00DEE8226E
:10176400A243923FC2431215A5EE2F60140E90803F
:1017740000E5216403121B1A6403121B1ADFF4DE52
:0B178400F21211EBC239A23F92432287
:1011EB00E524908002D2E4F07828121B14C2E4F0BC
:0511FB007828021B141E
:1015A5001215ACC3021969D3121969908000E5219F
:1015B500D2E1F07817121B14E524908002D2E1F0F5
:1015C500780C121B14C2E1F09080007812121B14E3
:0615D500E521F0D23922ED
:101A7600908000E5216403121B1A6403121B1ADF0F
:021A8600F42248
:0C1AF400908003E525C2E6F0D2E6F02267
:10196900E5264004D2E68002C2E6908004F0F5261E
:081979004001227805021B1455
:100EEF00907DC1E054F0B4F006121258020F71B4A5
:100EFF000005120D26806BB410051216118063B415
:100F0F002005121349805BB430051218038053B4C7
:100F1F0040051218B4804BB450051210688043B4CA
:100F2F006005121A88803BB470051215DB8033B44C
:100F3F008005120DC5802BB49005120F788023B455
:100F4F00A005121AC9801BB4B0051215318013B455
:100F5F00C005121934800BB4D00512193480031256
:090F6F000FF7907FC97400F02215
:051B20007406021936F5
:051B25007415021936E1
:101934007418C253753500901B4D858332858233EC
:0B194400F0A37400F0F52C752D0122BB
:10189200C253753500901B4D85833285823374A502
:1018A200F0A3E516F0540F240354FE03F52D752C16
:0218B200002212
:101A8800901B4F7462F5167402F0A37446F00218A6
:011A980092BB
:0F1ABA00901B4F7400F0A3F074E2F5160218921F
:10125800A3E0A3B403030213E1B40A030213DFB447
:101268000003021A99B4040302178FB4050302128B
:10127800FCB40603021395B407030217B7B40805B4
:10128800E0FF021A63B4090BE0FFA3E0FD12146D3E
:10129800021B20B40B03021B20B40D061215AC026E
:0312A8001B2022E6
:101A63001216AB901B4F74F2F5167408F0A3EFF047
:031A7300021892C4
:101A99001216DCE0F512FEA3E0F513FF050A021B9E
:011AA900201C
:1013DF00050A050A1216DCE0FEF512A3E0FFF5136D
:1013EF00C3E51D9420E51C9400500A204807E4B57E
:1013FF000A03021934D253907DC2E0B40302800372
:10140F00B40A0F7C00907DC7E0FD14250AF50A127F
:07141F0011348E2C8F2D22E9
:10178F007400F50AE51C451D601B30480F90800062
:10179F0078007900E030E104D8FAD9F8121AF4751C
:0817AF001C00751D00021B2047
:1012FC001216DCE0FCA3E0FDA3E0F8A3E0F9A3E008
:10130C00FAA3E0FB901B4CECF0E526D2E1D2E0BC5A
:10131C000306C2E0D2E18007BC0204C2E1D2E0F5D0
:10132C0026908004F0901B49EDF0901B4AE8F0A346
:0D133C00E9F0901B47EAF0A3EBF0021B2044
:1017B700907DC6E0FEA3E0FF907DC3E0B4000D304E
:1017C7003A05121764800D12186F80083038051219
:0717D7001A388000021B20FC
:10139500907DC4E0FF7E00A3A3A3E0FCA3E0FD12C3
:1013A5001134907DC3E0B40020303A08203905C2DD
:1013B500431215A57C07907DC1E0907DC9540FB4FB
:1013C5000802E0FC121194800E30380B203D031208
:0A13D50016451217DE8000021B20EF
:1016DC00907DC3E0B52E028022F52EB40006D24ACE
:1016EC007D40800BC24AB401047D2080027D107FB6
:0F16FC001012146D7DD87F0012146D907DC422E2
:100FF700A3E0A3C3B400028038B401028011B40295
:1010070002802FB403028008B40403021ABA22D361
:1010170012105D907DC6500CE584F8E0A3F608DF5A
:10102700FA021B20E0A30586F0A30586DFF6021B64
:1010370020D312105D901B4F7516E8500CE584F80D
:10104700E608F0A3DFFA0218920586E0A30586F00A
:10105700A3DFF6021892E0FFA3E0F584A3E0F5858D
:011067002266
:10170B00907F98E0C2E3F0C2E5F0F879C77B027AEC
:10171B0008E933F9E8C2E45002D2E4F0D2E3F0C2B4
:0D172B00E3F0DAEDEFF9DBE7E8D2E5F022BC
:10142600907F98E0C2E3F0C2E5F0FB79A77A08E97D
:1014360033F9EBC2E45002D2E4F0D2E3F0C2E3F0B7
:10144600DAED7828000000D8FB7A087F00907F9BB1
:10145600E0C372E2EF33FF907F98EBD2E3F0C2E392
:07146600F0DAEAD2E5F02202
:10146D00C2AF907F98E0D2E3F0908003E525D2E4FF
:10147D00F0F525EFF9907F98E0F87B027A08E933D3
:10148D00F9E8C2E45002D2E4F0C2E3F0D2E3F0DABC
:10149D00EDEDF9DBE7908003E525C2E4F0F525D20B
:0214AD00AF226C
:1014AF00C2AFE520907F97FA7809EAC2E6F0791E7D
:1014BF00D9FEEAD2E6F0D3EF00007907D9FE33CA9E
:1014CF004008C2E6F0CAD8F28006D2E6F0CAD8EADF
:1014DF00D2AF907F997A03E030E105D8FADAF8C3FA
:0114EF0022DA
:1016AB00907F96E020E0047E0180027E008E0CEF9E
:1016BB006009907F96E054FEF0800B907F96E0449B
:1016CB0001F0A23A9243E50C70047F0180027F0087
:0116DB0022EC
:100D2600C246907DC5E0540CF50CE030E42C907D75
:100D3600C3E0F539A3E0F53CE53854F34404F5384F
:100D4600D24CA3E030E603E4F50CE50C7047C24C48
:100D5600E53854F34408F538803B907DC2E0F50B46
:100D6600A3E0F511A3E0F517E53854FC4401F53886
:100D7600D24FE50C700AC24FE53854FC4402F538F0
:100D8600A23A9243C251C24E303A0AAF14EF6514EA
:100D960060FB1211EBE50CB40403121679E50CB4F2
:100DA600080312156B121B20C2AF907DC5E030E719
:0E0DB60006D23CD251D24EA251B39246D2AFD9
:010DC400220C
:10161100C246907DC2E030E014E538540C6020539E
:1016210038F3304C1A12156B43380C8012E53854DC
:1016310003600C5338FC304F0612156B433803D24C
:0416410046021B2022
:10134900C2AF907DC2E030E407E0A2E3925C80374F
:10135900C25CC256907DC3E0901B5DF0907DC2E0F7
:1013690030E10BA3E0F510E4901B44F08019907D67
:10137900C2E030E00CD256907DC4E0901B44F0806E
:0C13890006901B447401F0D2AF021B2040
:10180300E4901B4FF030560204F0901B5DE0901BF8
:1018130050F0A3E515F0A37480F0A3E53AF0751634
:0418230035021892E0
:1018B400C2AF907DC2E0F50DA3E0F508A3E0F50EFC
:1018C400A3E0F509C254A3E030E002D254D2AF023F
:0218D4001B20D7
:10106800121B20C2AF907DC2E0F50C7F02C28E90A9
:101078007DC4E0F4F58B907DC3E0F4F58DE58954EB
:101088000F4410F58953883FC28FC206907F97E5B9
:1010980020F0D28E308FFDDFD47F02D206907F976A
:1010A800E520F0C28E907DC6E0F4F58B907DC5E01A
:1010B800F4F58DC28FD28E308FFDDFDFD50CACE515
:0B10C80089540F4430F589C28ED2AF6E
:0110D30022FA
:1015DB00907DC2E02410547FF50CE030E715907D30
:1015EB00C4E0FFAD0C12184B901B4FEFF07516714A
:1015FB00021892907DC4E0FF907DC3E0FBAD0C120E
:06160B00000E121B20225C
:100DC500121B20907DC2E0FFC454C0F516E4901BB1
:100DD50043F0E516B44004D205801BE5167004C245
:100DE500058013E516B48008901B43743FF0800618
:100DF500901B43740FF0E538543F4516F538C2048F
:100E0500907DC2E030E402D204907F97E520F09017
:100E15007DC2E05403F516B40103121679E516B444
:100E2500020312156BE516B40303120E5C907DC226
:100E3500E0FFC4135403F51664016005E516B40319
:100E450008C217908010E522F0E516B40208D21703
:070E5500908010E522F0225D
:100F7800C2AFE53854CF901B4FF0305A04E044100C
:100F8800F0305807901B4FE04420F0305707901B73
:100F98004FE04430F0A204E433901B50F0907F9966
:100FA800E020E107901B50E04404F0301707901B45
:100FB80050E04408F0E50D6007901B50E04410F045
:100FC800E5086007901B50E04420F0E50E600790AC
:100FD8001B50E04440F0E5096007901B50E0448056
:0F0FE800F0901B51E530F0D2AF751693021892BE
:10153100907DC2E0F50CE4F516F50C907DC2E0FF5C
:10154100E50CC39F501874C3250CF582E4347DF576
:1015510083E0FF1214AF50020516050C80DD901BCD
:0A1561004FE516F07516B10218925E
:0F1AC900121B20C23E907DC2E030E002D23E22CE
:1010D4001201000100000040970D0101020001020D
:1010E400000109022000010100A00009040000021F
:1010F400FF000000070582024000000705020240CD
:101104000000040309040A03530042004900470095
:101114001E035500530042002D00430041004D00C2
:10112400200045006E00670069006E006500000045
:041B2E0001020408A4
:10030E00901B6812116300000000C25EC23BC25512
:10031E00C2401208AD7E107FD48E188F19751A1038
:10032E00751BE6751E11751F06EE54E07003020470
:10033E0072901B6CE4F0A37480F0A3EEF0A3EFF0C8
:10034E00C374329FFF74119ECF2402CF3400FEE49B
:10035E00FCFD901B64121157901B5E12116300007E
:10036E000000901B64E0FCA3E0FDA3E0FEA3E0FF11
:10037E00901B5EE0F8A3E0F9A3E0FAA3E0FBC31242
:10038E001146503A901B60E0FEA3E0FF901B6CE01C
:10039E00FCA3E02FF582EC3EF58374CDF0901B5E4E
:1003AE00E0FCA3E0FDA3E0FEA3E02401FFE43EFE9B
:1003BE00E43DFDE43CFC901B5E12115780A4901BA3
:1003CE005E12116300000000901B64E0FCA3E0FDD0
:1003DE00A3E0FEA3E0FF901B5EE0F8A3E0F9A3E02C
:1003EE00FAA3E0FBC31211465049901B60E0FEA336
:1003FE00E0FF901B6EE0FCA3E02FF582EC3EF58350
:10040E00E0FD901B6CE0FAA3E02FF582EA3EF58347
:10041E00EDF0901B5EE0FCA3E0FDA3E0FEA3E02464
:10042E0001FFE43EFEE43DFDE43CFC901B5E121138
:10043E00578095901B6CE0F518A3E0F51974D42441
:10044E0080FF741034FFFE901B62F0A3EFF0C3E543
:10045E001B9FF51BE51A9EF51AC3E51F9FF51FE5B9
:10046E001E9EF51ED2E843D820907F95E044C0F042
:10047E00907FAFE04401F0907FAEE0441DF0907F9E
:10048E00ADE04404F0D2AF120732204052204005B6
:10049E00D25F1212AB901B68121163000000007F36
:1004AE00407E927D047C00901B68E0F8A3E0F9A3E7
:1004BE00E0FAA3E0FBC312114650CF2040CC901BB4
:1004CE0068E0FCA3E0FDA3E0FEA3E02401FFE43E10
:1004DE00FEE43DFDE43CFC901B6812115780C0E524
:1004EE008E54F84401F58E304005120523C240307B
:1004FE005E12C25E1218F8203B07907FD6E020E70E
:10050E00F312194F120C59120C59120C59120C5994
:05051E00120C5980D20F
:10052300907FE9E07003020602147003020665245B
:10053300FE70030206D424FB70030205FC1470034F
:100543000205F61470030205EA1470030205F02491
:10055300056003020723907FEBE024FE601614601E
:100563004224027078E518907FD4F0E519907FD586
:10057300F002072A907FEAE0FF1214F0AA06A90707
:100583007B018B3D8A3E893FEA49600DEE907FD423
:10059300F0EF907FD5F002072A907FB4E04401F09A
:1005A30002072A907FEAE0FF121738AA06A9077B01
:1005B300018B3D8A3E893FEA496018EE907FD4F073
:1005C300EF907FD5F0E4907FB5F0907FB47402F0A4
:1005D30002072A907FB4E04401F002072A907FB417
:1005E300E04401F002072A121AE602072A121B0C42
:1005F30002072A12000302072A121AD802072A90B6
:100603007FE8E0247F601A14601E2402704AA23B34
:10061300E433FF25E0FFA255E4334F907F00F080E1
:1006230029E4907F00F08022907FECE0F45480FF77
:10063300C4540FFFE054072F25E024B4F582E434BB
:100643007FF583E05401907F00F0E4907F01F09008
:100653007FB57402F002072A907FB4E04401F002F0
:10066300072A907FE8E024FE601D2402600302074E
:100673002A907FEAE0B40105C23B02072A907FB4C7
:10068300E04401F002072A907FEAE0703B907FECA0
:10069300E0F45480FFC4540FFFE054072F25E024F7
:1006A300B4F582E4347FF583E4F0907FECE054808A
:0F06B300FF131313541FFFE054072F907FD7F04E
:0306C200E4F5401C
:1006C500E04420F0805F907FB4E04401F0805690D4
:1006D5007FE8E024FE60182402704A907FEAE0B4C7
:1006E5000104D23B803F907FB4E04401F080369016
:1006F5007FEAE07020907FECE0F45480FFC4540F53
:10070500FFE054072F25E024B4F582E4347FF58318
:100715007401F08010907FB4E04401F08007907F71
:0C072500B4E04401F0907FB4E04402F026
:0107310022A5
:03003300021B2A83
:041B2A0053D8EF326B
:0D00360000170B0907070605090A0A0CFF51
:10182700052F7E00E52F5403242EF582EE341BF599
:1018370083E493FFE52554F0FEEF4EF525908003F2
:04184700E525F02281
:100E5C00901B437403F0C249D22F908003E525F018
:100E6C00E4F516F5367530FF7D64E516C3947050C5
:100E7C004812182785140CC3E514950CC39D40F734
:100E8C007D05E5366013FF0536EFC3940340DBE5C3
:100E9C002F20E0D67530098020908000E013925A04
:100EAC00AF160516EFC3940C4008304405305A02B7
:100EBC000536A25AB3924480B1532FFED25AC24483
:100ECC00C258C2577536FFD249C22F908003E52510
:100EDC00F0E53670FCE4901B43F0D205907F97E56B
:020EEC0020F0F4
:010EEE0022E1
:10167900C249305704D25B8026C25B305A21D25806
:10168900C25AE52F5403901B2E93FFE52554F0FE13
:10169900EF4EF525908003E525F0E4F536F537D2D0
:0216A9004922D4
:10156B00C249305804D24D802EC24D304429D25737
:10157B00C244C207907F97E520F0E52F5403901BE0
:10158B002E93FFE52554F0FEEF4EF525908003E5F5
:0A159B0025F0E4F536F537D24922B9
:03000B00020046AA
:10004600C0E0C0F0C083C082C0D075D000C000C080
:0D00560001C002C003C004C005C006C00701
:10006300901B42E004F0E0540760030202CA2049F7
:100073000302012F20580620570302011F20570FA8
:10008300E537700B901B45E06409600302012FE51F
:10009300367071908000E0139245E5377005750F57
:1000A300FF801C302F19A245304201B35011305844
:1000B3000830420B85370F800620420385370FC275
:1000C3002FA24592421218270537E5379000369341
:1000D300F536E537640C7054908003E525F0850F01
:1000E30030305814D244C258D207907F97E520F09D
:1000F300304D3912156B8034D25AC257305B2D12F2
:10010300167980281536E536B40121E537C39407FF
:10011300401AD22F908003E525F08010E536600C5D
:10012300D536095325F0908003E525F0303E75C29E
:1001330036908004E526F09080027401F0741DF07F
:100143007419F09080007474F0908001747FF075DE
:100153003D04908000748FF09080017441F0908092
:10016300027419F0D53DEB753D04908001E4F090E5
:1001730080027410F0D53DF29080007474F090808A
:1001830001747FF09080027401F0908000E521F00B
:10019300908001E523F0908002E524F0D236908030
:1001A30004E526F0305117303C07C23C1211EB80B6
:1001B3000DAF171517EF7006C251D2468063901B1F
:1001C30045E004F0E0640A60030202CAF00514E5A6
:1001D300147006901B46E004F0D25020460302023E
:1001E30073E5385403FFBF0108205A033044020566
:1001F30038E5385403FFBF021DAF171517EF70160C
:10020300AF111511EF700FAF0B150BEF7008304FD7
:100213001012156B0538E5385403FFBF030E305A2F
:100223000B304E05C2431215A55338FCE538540C68
:10023300FFBF040C204403305A0674042538F538F4
:10024300E538540CFFBF081AAF3C153CEF7013AFF1
:10025300391539EF700C304C1412156B74042538B2
:10026300F538E538540CFFBF0C06305A035338F306
:10027300305406E514540F7035753D00E50D6005E7
:10028300433D01150DE5086005433D021508E50EE4
:100293006005433D04150EE5096005433D08150956
:1002A300E52054F0453DF520907F97E520F0901B25
:1002B30043E0FF600655147002B205907F97E52076
:1002C300F0E514543F600330592630432330522065
:1002D300E53B6407601AB208B209908000E521F09B
:1002E300753D04D53DFDB208B209908000E521F0CB
:1002F300D007D006D005D004D003D002D001D0005F
:0B030300D0D0D082D083D0F0D0E03208
:101AAA00040103000505000301000200FFFFFEFE1A
:1008AD00D23B907F92E054FDF0E4907FE2F0F5862C
:1008BD00907F9574C3F0907F9E74FBF0907F93743E
:1008CD0028F0E4907F94F0907F9C747DF0907F965B
:1008DD007401F0907F9D74FFF0907F977430F090CD
:1008ED007FDD7409F0907FA1E04401F0907FB27438
:1008FD0000F0A37446F0907FAFE04406F0758C06CF
:10090D00E58954F84402F589538EF7D28CD2A97536
:10091D002560908003E525F0AF3A12170BD20690B3
:10092D007F97E520F0753840D246D2527524017577
:10093D00217475237F752603908000E521F090804A
:10094D0001E523F0908002E524F0908004E526F087
:10095D00908010E522F0901B497401F07D0C7F40D2
:10096D0012146DE4FD7F7012146D7DD8E4FF121426
:10097D006D7D407F1012146DD24A7D0C7F201214B4
:10098D006D7D1E7F5012146D7D1E7F3012146DE42F
:06099D00FD7F6002146DF5
:10073200908006E4F0A3740AF0908008E4F0A374B9
:1007420009F090800AE4F0A304F0D236908004E528
:1007520026F0D237E526F085140C908000E030E1D7
:100762000AC3E514950CD3940A40EF121AF4120E40
:100772005C7F011216AB753404E4901B4AF0A3F0BF
:10078200750C02E50C2410FD7FA012184B901B4B38
:10079200E02FF0901B4AE03400F0050CE50CC39406
:1007A2002040E07D117FA012184BEFFE901B4BE022
:1007B2002400F0901B4AE03EF07D107FA012184BFF
:1007C200901B4BE02FF0901B4AE03400F0E0F470F5
:1007D20003A3E0F470297D137FA012184B8F347DA0
:1007E200167FA012184B8F0D7D1A7FA012184B8F07
:1007F2000E7D247FA012184B8F0CE50C139238E566
:100802003424FB601924FB601A24FE601B1460254B
:1008120014602C24FC60238000753118802A753105
:100822003080257531108020753146D23590800494
:10083200E526F08013753120800E753142800375F4
:100842003134D23AD208D243E50C30E50A901B5D2E
:10085200746FF0D2568008121426901B5DEFF0E4FC
:10086200F50CE50EC394804003750C01E50C245091
:10087200FFE50E25E0FD12146DE4F50CE50DC394C1
:10088200804003750C01E50C2460FFE50D25E0FDB9
:1008920012146DE4F50EF50DA2389232908004E543
:0A08A20026F0D204907F97E520F0C5
:0108AC002229
:100A8E001214268F15205603020B36E4FD901B5DC3
:100A9E00E0FCC3951540027DFFE514547FFFBF04B3
:100AAE0017ED600C901B44E0F4600DE004F080083C
:100ABE00901B44E0600214F0E5145407707CED6066
:100ACE0030ECC39515F53EE49400F53DE53EAE3DA4
:100ADE007803C333CE33CED8F9F53E8E3D901B440A
:100AEE00E0FB7E00253EEE353D7039EB253EFD8068
:100AFE0033ECFFE515C39FF53EE49400F53DE53E6E
:100B0E00AE3D7803C333CE33CED8F9F53E8E3D904D
:100B1E001B44E0FFFBC3E53E9BE53D94005005C33F
:100B2E00EF953EFD8D108012901B44E0600CE51495
:100B3E0054077006E51060021510E510D3953A4083
:100B4E0002053AE510C3953A5002153AAF3A12171C
:100B5E000BE53A600AD216908010E522F08008C2AA
:090B6E0016908010E522F0C2503F
:010B7700225B
:100C5900305D3F907DC0E0F50CA3E0FFC4540FF573
:100C690016E50CB4A509E516901AAA93B4FF051266
:100C79001934801CE516901AAA93FF907DC1E0549F
:100C89000F6F6004EFB4FE05120EEF8003121B25EF
:100C9900C25D30532FE535702BC3E52D951DE52C2D
:100CA900951C5011E52DAE2C7805CEC313CE13D863
:100CB900F9F535800FE51DAE1C7805CEC313CE13AB
:100CC900D8F9F535538EF8120B78058E30480F1286
:100CD90009A3A24792475021C248C247801BE50A8F
:100CE9006017E51D2513FFE51C3512FED3EF9400AF
:100CF900EE94105004D248150A305006205C0312B5
:100D09000A8EE5385403FFBF0210E511D394005051
:0D0D190006E50B94004003C25922D2592276
:08000300907FEAE0F544D322EE
:0E1AD800907F00E544F0907FB57401F0D322BA
:081B0C00907FEAE0F543D322CB
:0E1AE600907F00E543F0907FB57401F0D322AD
:10198100C0E0C083C082D2405391EF907FAB74011D
:08199100F0D082D083D0E032D7
:1019E000C0E0C083C0825391EF907FAB7404F0D00D
:0619F00082D083D0E0323A
:1019F600C0E0C083C0825391EF907FAB7402F0D0F9
:061A060082D083D0E03223
:101A0C00C0E0C083C0825391EF907FAB7410F0D0D4
:061A1C0082D083D0E0320D
:10199900C0E0C083C082D25E5391EF907FAB7408E0
:0819A900F0D082D083D0E032BF
:1019B100C0E0C083C082D25D5391EF907FAA7404CE
:0819C100F0D082D083D0E032A7
:100B7800907FB8E020E114E53560081535792078D4
:100B8800208026E52D7005E52C7001227820E52DC2
:100B9800C398E52C94005002A82DE8F9305370E56D
:100BA8001DC398E51C940040E2907FE27450F074F5
:100BB80000907FE4F0747E907FE3F0907FE57420EE
:100BC80098702C7802C2AFF0F0F0F0F0F0F0F0F08E
:100BD800F0F0F0F0F0F0F0F0F0F0F0F0F0F0F0F00D
:100BE800F0F0F0F0F0F0F0D8DED2AF8008C2AFF04D
:100BF800F0D8FCD2AF907FE27400F0907FB9E92979
:100C0800F0C3E51D99F51DE51C9400F51C802F85A2
:100C180033848532857400907FE4F0747E907FE39E
:100C2800F0907FE5C2AF0586E0A30586F00586E073
:100C3800A30586F0D8F0D2AF907FB9E929F0858472
:100C480033858532E52DC399F52DE52C9400F52CD7
:010C58002279
:011B3400327E
:1009A300E53B24F97003020A5924076003020A8D08
:1009B300204803020A8DC2AFC237908004E526F0B7
:1009C3007F05121B32C236908004E526F0304A259B
:1009D300303A18C243304E09E534641260031211F1
:1009E300EB901B49E0FF121A768015901B49E0FF3C
:1009F300121919800B303808901B49E0FF121A2294
:100A0300901B4AE0FEA3E0FF8E45F546901B47E0AE
:100A1300FCA3E0FDEF2DFBEE3CCB2513F546EB35B8
:100A230012F545908006F0A3E546F0C39FF546E531
:100A3300459EF545908008F0A3E546F090800AECCA
:100A4300F0A3EDF0D236908004E526F0D237E52608
:100A5300F0D2AF753B07908000E020E12DE5132530
:100A63001DF51DE512351CF51CE50A6018E51D256D
:100A730013FFE51C3512FED3EF9400EE94105005DE
:0A0A8300150A0209B9E4F53BD24759
:010A8D002246
:101A4E00C3907FA57800E020E003D8FA2220E2FCC4
:051A5E0030E1F9D32284
:1018D600C2AF907FA57480F0907FA6EF54FEF01201
:1018E6001A4E500D7400F0907FA6EDF0121A4E506D
:0218F6000022CE
:10000E001218D65009907FA6EBF0121A4EC3907FAD
:10001E00A57440F05008907FA6E0FF907FA5E020E9
:05002E00E6FCD2AF2248
:10184B001218D6501B7480F0907FA6EF54FE440103
:10185B00F0121A4E500A7420F0907FA6E0121A4E26
:04186B00D302001C88
:101A2200908001E523C2E4F06403C2E4F0D2E4F062
:061A3200DFF8E523F022BD
:1017DE00EF2E601DD3121969908001E5230E64105F
:1017EE00F0640BF06410F0640BF0DFF2DEF0E52332
:0517FE00F0C3021969AF
:101A3800908002E524D2E3F07805121B14C2E3F08B
:061A4800121645C23D220A
:10164500908001E5237D7D7C0B7B10C2AF6BF06C38
:10165500F06BF06CF06BF06CF06BF06CF06BF06CA9
:10166500F06BF06CF06BF06CF06BF06CF0DDDED2D3
:04167500AFD23D2291
:10194F00907FD6E030E712E04401F07F147E001262
:0A195F0019C9907FD6E054FEF02273
:1018F800907FD6E04480F04387010000000000227A
:0712AB00907FD6E04408F03B
:0312B200E4F53D23
:0412B500E054FBF016
:0312B900E4F53D1C
:1012BC00E04408F0305F04E04402F07FDC7E05126D
:1012CC0019C9907F92E030E3077FDC7E051219C9C3
:1012DC00907FAB74FFF0907FA9F0907FAAF05391B0
:0812EC00EF907FD6E054F7F00B
:0312F400E4F53DE1
:0512F700E04404F022B8
:02173800A907FF
:10173A00AE1EAF1F8F828E83A3E064037017AD01C4
:10174A0019ED7001228F828E83E07C002FFDEC3E22
:09175A00FEAF0580DF7E007F0078
:011763002263
:0214F000AD0746
:1014F200E4FCAE1AAF1B8F828E83A3E06402702AD3
:10150200AB040CEBB50501228F828E83A3A3E0FA14
:10151200A3E08A41F5426241E5416242E54262410D
:0E1522002FFBE5413EFEAF0380CC7E007F0034
:011530002298
:1019C9008E3E8F3FE53F153FAE3E7002153E4E609D
:0719D9000512190880EE223F
:101908007400F58690FDA57C05A3E582458370F9F2
:0119180022AC
:03004300021200A6
:10120000021981000219F6000219E0000219990082
:10121000021A0C00021B3400021B3400021B3400B3
:10122000021B3400021B3400021B34000219B100FF
:10123000021B3400021B3400021B3400021B34006A
:10124000021B3400021B3400021B3400021B34005A
:08125000021B3400021B3400F4
:03000000021B00E0
:0C1B0000787FE4F6D8FD75814602030EE4
:10113400EF8DF0A4A8F0CF8CF0A428CE8DF0A42ECF
:02114400FE2289
:10114600EB9FF5F0EA9E42F0E99D42F0E89C45F0FF
:011156002276
:0C115700ECF0A3EDF0A3EEF0A3EFF0220B
:10116300A8828583F0D083D08212117A12117A1269
:10117300117A12117AE473E493A3C583C5F0C5838E
:10118300C8C582C8F0A3C583C5F0C583C8C582C8D6
:011193002239
:00000001FF
